:06000000008077022EA52E
:03000B0002259F2C
:030013000224794B
:03001B0002269B1F
:03002300022E4B5F
:10002B003202534D50544520496E746572666163BC
:10003B0065202020286329203139393520202041A3
:10004B006C636F726E204D63427269646520496EFA
:10005B00632E2020200D534D50544520496E74655E
:10006B00726661636520432056362E30380D00C210
:10007B00AF75D00075816C43B0FF4390FF7589213C
:10008B00758804758DFD758BFDD28E7589237598DA
:10009B00D0787FE4F6D8FD751800751E149000001B
:1000AB007400F0A3A883B820F974FF90E800F090D7
:1000BB001523F090E000F0901522F075A015781E36
:1000CB0090E000E0F20890E800E0F2C294D296755E
:1000DB0066057401904002F0D297901522E044100F
:1000EB00F090E000F0120218903017120295903049
:1000FB002A120295121D281222AC1222599080024C
:10010B0074B5F0122FAE30B5FD20B5FDC294122F91
:10011B00BC30B5FD20B5FDD2947400904002F012B6
:10012B002FBC30B5FD20B5FDC294122FBC30B5FDF0
:10013B0020B5FDD294122FBC7401904002F030B563
:10014B00FD20B5FDC294122FBC30B5FD20B5FDD2FC
:10015B0094122FBC30B5FD20B5FDC294122FBC30CC
:10016B00B5FD20B5FDD294122FAE122FAE122FAECD
:10017B00122FAE122FAE122FAE122FAE122FAE12B7
:10018B002FAE122FAE122FAE90303D12029575B8D6
:10019B000075A811D2AF751296901522E054FBF0A2
:1001AB0090E000F01215D01216471216E5C215C2D8
:1001BB003FD201302A04C201C22C75816C3001443C
:1001CB00C28CC292758A00754C00C204D246D28C86
:1001DB00D2A990301712029590303D12029512055C
:1001EB006F302303120CA23001121203323004EED3
:1001FB00C204B2941207CA30010280E2C28CC2A9B7
:10020B00C246D2922022030217DD021A747A3012F0
:10021B00023C7A3012023C7A3812023C7A8012028B
:10022B003C7A0612023C7A0C12023C7A0112023C16
:10023B0022C0F075F00075A0A07802E230E707004D
:10024B00D5F0F30202557800EAF2D0F022C0F07537
:10025B00F00075A0A07802E230E70700D5F0F302BA
:10026B00027475A0A07801EAF2D0F022C0F075F00C
:10027B000075A0A07802E230E70700D5F0F3020288
:10028B009275A0A07803E2D0F022740093A312021F
:10029B00B3FA740093A32AFA12023C740093A3607E
:1002AB0006FA12025880F42283227FBF93D37A85F9
:1002BB0012023CE55175F000600475F00A8424309D
:1002CB00FA120258E5F02430FA1202587A3A120266
:1002DB0058E55275F000600475F00A842430FA1268
:1002EB000258E5F02430FA1202587A3A120258E515
:1002FB005375F000600475F00A842430FA1202582A
:10030B00E5F02430FA1202587A2E120258E5547591
:10031B00F000600475F00A842430FA120258E5F0FC
:10032B002430FA12025822303A08E56930E0031201
:10033B000356303B08E56930E10312048D303C086D
:10034B00E56930E203120490C23A22E562C395617B
:10035B00F4B41200500302048CA86275A01C74FE46
:10036B00F2F5F075A01B7401F20875A01CE56BF299
:10037B0025F0F5F075A01BE4F20875A01C7428F2AB
:10038B0025F0F5F075A01BE4F20875A01CE56AF2E8
:10039B0025F0F5F075A01BE4F20875A01CE551F2F1
:1003AB0025F0F5F075A01BE4F20875A01CE5F0C371
:1003BB0013F275A01B7401F20875A01C74FEF2F504
:1003CB00F075A01B7401F20875A01CE56BF225F00B
:1003DB00F5F075A01BE4F20875A01C7428F225F04B
:1003EB00F5F075A01BE4F20875A01CE56A2401F278
:1003FB0025F0F5F075A01BE4F20875A01CE552F290
:10040B0025F0F5F075A01BE4F20875A01CE5F0C310
:10041B0013F275A01B7401F20875A01C74FEF2F5A3
:10042B00F075A01B7401F20875A01CE56BF225F0AA
:10043B00F5F075A01BE4F20875A01C7428F225F0EA
:10044B00F5F075A01BE4F20875A01CE56A2402F216
:10045B0025F0F5F075A01BE4F20875A01CE553F22E
:10046B0025F0F5F075A01BE4F20875A01CE5F0C3B0
:10047B0013F275A01B7401F2088862906005740674
:10048B00F022C23B22E562C39561F4B40C00500329
:10049B0002056EA86275A01C74FEF2F5F075A01B28
:1004AB007401F20875A01CE56BF225F0F5F075A050
:1004BB001BE4F20875A01C7428F225F0F5F075A06A
:1004CB001BE4F20875A01CE56A2404F225F0F5F094
:1004DB0075A01BE4F20875A01C901563E0F225F0E3
:1004EB00F5F075A01BE4F20875A01CE5F0C313F240
:1004FB0075A01B7401F20875A01C74FEF2F5F07563
:10050B00A01B7401F20875A01CE56BF225F0F5F049
:10051B0075A01BE4F20875A01C7428F225F0F5F009
:10052B0075A01BE4F20875A01CE56A2405F225F002
:10053B00F5F075A01BE4F20875A01C901564E0F2B1
:10054B0025F0F5F075A01BE4F20875A01CE5F0C3CF
:10055B0013F275A01B7401F2088862906005740693
:10056B00F0C23C22E559655A60081205A2202326E9
:10057B0080F2302D051229B5800EE56365646008A5
:10058B001206C820231080F2E55F65606008120632
:10059B00F380F585605F2275A01EA959E3FA75A05B
:1005AB001DE3FB0559C239C229BB0006EA20280FFF
:1005BB00803CEA30E73690155CF0D2280206C7C2C1
:1005CB0028B4FE0DF51CF51D751800751E140206DA
:1005DB00C7B480005005751D00805E751DFDD224CB
:1005EB0090155DC0E0E4F0D0E0020684D229AD1D89
:1005FB00BDFE03020610BD0003020660BDFD030233
:10060B0006840206C7BB0002801AF5F090155CE069
:10061B00251CC313B5F005D2230206C77455121758
:10062B00B20206C7851EA0A818F2251CF51C088867
:10063B0018B80002051E0206C790155CE075831CF6
:10064B00856282F0740175831BF00582E56165821A
:10065B00602485826220391E75831C856282EAF0D4
:10066B00EB75831BF00582E561658260098582620B
:10067B009060057406F00206C730290990155DE0FD
:10068B00C313FAC22990155DE02AF0758318855EB5
:10069B0082EAF0302406C224740180027400758350
:1006AB0017F00582E55D6582600F85825E908002A2
:1006BB0074B5F09080057406F00206C72275A01A77
:1006CB00A963E3FA75A019E3FB056375831F855CCA
:1006DB0082EAF00582E55B6582600385825C2020FF
:1006EB0002D299D2390205B275A016A85FE2055F56
:1006FB00B4FE0BD230C231C232C2330207C9303022
:10070B000AB41302D231C2300207C9303110B420FF
:10071B0000505F901563F0C231D2320207C93032FC
:10072B000B901564F0C232D2330207C930334BF849
:10073B007A11901563E02AFA901564E02A547FC36E
:10074B0098702F901564E0F8901563E0901565256F
:10075B0082F58274003583F583E8F0D23C30E504F2
:10076B00D234800375671E901522E054FDF090E0A3
:10077B0000F0C231C232C2338044C231C232C23302
:10078B00F5F0B4FF0B2020FD7598D8752C00D22CFA
:10079B00302C12052C7405B52C0B2020FD7598D828
:1007AB00752C00D22CE5F075831F855C82F00582D9
:1007BB00E55B6582600385825C202002D299222052
:1007CB0090187566057401904002F0D2979015222F
:1007DB00E04410F090E000F08016D56613740090A2
:1007EB004002F0C297901522E054EFF090E000F039
:1007FB0020930F203719D23774BF75F00A12176583
:10080B00800D30370AC23774BF75F00B1217657540
:10081B00A015791FE3FB90E800E0F36B5B60357B81
:10082B000833502EC0E090E000E030E61C75F0007D
:10083B0030E70375F01020E50343F04074B12BFA59
:10084B00EBF9122007D0E0800974B12BFA12208F3C
:10085B00D0E0DBCD75A015781EE2FA90E000E0F257
:10086B006A5AFAEA541F606330E029D291C2012020
:10087B001510200019C23F302214301F11121C59C1
:10088B00800C103F028007C2AF121C59D2AFC200BE
:10089B00C215803730E109202B06D200C291802B84
:1008AB0030E308C2AFD215D2AF802030221530E42E
:1008BB0006C2AFD215D2AF30E211D201D2911220C3
:1008CB00DB800830E205D2011220DB227851E608EA
:1008DB00460846084660121208F57002800B120992
:1008EB008260067D16DDFE80F522900000E060261A
:1008FB00F975650030257D20267A7E107F008E826B
:10090B008F83E0B4FF02806CF5F07851E6B5F0020E
:10091B0080104060D902805C74082EFEEF3400FF1B
:10092B0080DCA3E0B4FF02804BF5F008E6B5F002E3
:10093B008004404080DEA3E0B4FF028037F5F0086E
:10094B00E6B5F0028004402C80CAA3E0B4FF02801D
:10095B0023F5F008E6B5F0028004401880B6E56593
:10096B00B4000DA3AB82AC83901520EBF0A3ECF09D
:10097B00056580A0E56522901520E0FBA3E0FCE572
:10098B0065B400030209CC8B828C83E0FEA3E0FFED
:10099B00A3E0F970030209BBA3E0B4FF030209CF84
:1009AB00B4800050030209FE020A59D5650280117A
:1009BB00EB2408FB901520F0A3EC3400FCF00209AB
:1009CB0092E56522E55CC3955BF489F0B5F00050C8
:1009DB00030209CC8E828F83A85C75A01FE0F2A363
:1009EB0008D9FA885C202002D299D565030209CC7C
:1009FB000209BBE562C39561F489F0B5F0005003C1
:100A0B000209CC8E828F83A86275A01CE0D2E7F21C
:100A1B0075A01B7401F2D903088022A308D90280A8
:100A2B000FE075A01CF275A01B7400F2A308D9F19E
:100A3B00E075A01CF275A01B7401F2A308886290EC
:100A4B0060057406F0D565030209CC0209BBE55EAF
:100A5B00C3955DF489F0B5F00050030209CC8E828A
:100A6B008F83A85EE075A018F275A0177401F2A32E
:100A7B0008D9030209BBE075A018F275A017740022
:100A8B00F2A308D9F1885E90800274B5F0908005CE
:100A9B007406F0D565030209CC0209BBE538C454D2
:100AAB000FF5F0E53954F045F030E72530E62254E8
:100ABB003FF5F0B43F028024900007E0B5F00280D0
:100ACB001B901500E0600AFAA3E0B5F002800DDA86
:100ADB00F790153EE4F0A3F0A3F08008901536E5EF
:100AEB00F0F0D21622901536E0F5F0A3E53AC45497
:100AFB000FF9E53B543049F025F0F5F0A3E53CC484
:100B0B00540FF9E53D543049F025F0543FF5F09082
:100B1B001536E5F0F022901536E0F5F0E53EC454BD
:100B2B000FF9E53F543049B5F002800B90153EE4C8
:100B3B00F0A3F0A3F08020C21E7903783E75A015B8
:100B4B00E2F5F0E0B5F0028002D21EF2121F84D95A
:100B5B00EF301E03021F8C227400B5520DB5530AE1
:100B6B00B551077403B55400500122901526E0606F
:100B7B00F9FA7400F0A3A85E122252B4030040F8F5
:100B8B0075A018E0D2E7F2FB75A0177401F2087597
:100B9B00A0187408F22BFB75A0177400F20875A04F
:100BAB0018EBF275A0177400F208885E75A08079B7
:100BBB000274B5F375A08079057406F3A3DAB9C294
:100BCB001B22900000E07005D226020C2675F00067
:100BDB00900005E0C395F0900003F075F0089000CD
:100BEB0006E095F0900004F0900000E0C226C3945C
:100BFB00025002802604FA7505137504008504065D
:100C0B008505077907120C98EAFB120C2979071254
:100C1B000C98DBF67905120C98DAE2D22522C08209
:100C2B00C083A8058504A0850782850683E0F5F0BF
:100C3B00E2C395F0C0D0120C70E0F5F0E2D0D09585
:100C4B00F0C0D0120C70E0F5F0E2D0D095F0C0D02F
:100C5B00120C70E0F5F0E2D0D095F04003120C844A
:100C6B00D083D08222C0E01582E582B4FF021583C7
:100C7B0018B8FF0215A0D0E0227908E2F5F0E0F2F7
:100C8B00E5F0F0A308B8000205A0D9EF22E724088D
:100C9B00F719E73400F722901400E0B44203020E78
:100CAB00EA543F2323900CB473020DBC00020FD502
:100CBB000002107600021087000210A400020DB48F
:100CCB00000210B8000210DE00021118000211AE73
:100CDB00000213A1000213C5000213EB000214055E
:100CEB000002141100021464000214C30002159CCC
:100CFB000002157800021552000215290002113D61
:100D0B000002115D0002132200021444000214536E
:100D1B000002139000020DB400020DB400020DB4DA
:100D2B0000020DB400020DB400020DB400020DB4AC
:100D3B0000020DB400020DB400020DB400020DB49C
:100D4B0000020DB400020DB400020DB400020DB48C
:100D5B0000020DB400020DB400020DB400020DB47C
:100D6B0000020DB400020DB400020DB400020DB46C
:100D7B0000020DB400020DB400020DB400020DB45C
:100D8B0000020DB400020DB400020DB400020DB44C
:100D9B0000020DB400020DB400020DB400020DB43C
:100DAB0000020DB400020DB40074551217B2C22329
:100DBB0022901401E0B4FE03020DE0B4FF03020E17
:100DCB000EB40003020E0EB4FD03020E0E74551288
:100DDB0017B2C22322120DEB74AA1217B2C223222E
:100DEB007A079000007400F0A3DAFCD226D22575A6
:100DFB001800751E14751F007400900005F0740820
:100E0B00A3F022C21EF5F0202606900000E070032E
:100E1B00020ED9FBF51F7A01A9F0EA75F008A4249C
:100E2B000FF582E5F03400F58389F0E0B5F0028030
:100E3B0003020ECCD21EE582C39403F582E58394A4
:100E4B0000F583E0FCA3E0FDA3E0F9E51FC39A04E2
:100E5B00C0F075F008A4AFF0FEEA1475F008A424F6
:100E6B0010F8E5F03400F5A0EA75F008A42410F5AD
:100E7B0082E5F03400F583120F10ECF8EDF5A0E9E4
:100E8B002CF58274003DF5837400C39582FE7414B7
:100E9B009583FF120F10900003E0C399F0A3E09429
:100EAB0000F0A3E0C399F0A3E09400F0120F1FD061
:100EBB00F01B151FE51FB40003020DE0BB000C80F7
:100ECB000D0ABB00028007DB028003020E23301EDB
:100EDB0006E51F900000F074AA1217B2C22322A8D5
:100EEB005C9000617900E993601175A01FF209080D
:100EFB00E8B55BF22020FAD29980F6885C202002BC
:100F0B00D299C22322E0F2121F84DEF9BF000280C5
:100F1B0002DFF222900014E51F6029F8E0C39CAEBB
:100F2B0082AF83A3E09505400D8E828F83E0C3993A
:100F3B00F0A3E09400F074072582F58274003583EA
:100F4B00F583D8D822900000E0F5F0FA7B007E0DF7
:100F5B00900003E02AFA74003BFBA3DEF69000102E
:100F6B00AEF0BE0003020F817F08E02AFA74003B4B
:100F7B00FBA3DFF6DEF2900003E0FFA3E0FE900898
:100F8B0000EE4F600FE02AFA74003BFBA31FBFFF7C
:100F9B00F01E80ED7E0F901500E02AFA74003BFBEB
:100FAB00A3DEF67E0F90150FE02AFA74003BFBA32D
:100FBB00DEF67E20901546E02AFA74003BFBA3DE9A
:100FCB00F6900001EAF0A3EBF022900000E004B4ED
:100FDB00FE0874551217B2021073F014F5F0740872
:100FEB00A42410F8E5F03400F5A07A04901401E085
:100FFB00F2121F84DAF9E0B4FE0E900000E014F058
:10100B0074551217B2021073FDA3E0FCA3A982AAB8
:10101B0083900003E02CF0A3E03400F0900005E097
:10102B00F5F0F2121F84E0F2FB121F84ECF2121F98
:10103B0084EDF2121F8474FFF2121F84F2121F84CC
:10104B00F2121F84F28A838982A9F0E08BA0F3A3AA
:10105B0009B900010BDCF4900005E9F0A3EBF0C239
:10106B0026C22574AA1217B2C223222026062025D7
:10107B0003120BCD74AA1217B2C22322121EF974DB
:10108B00AA1217B2C22320340B901522E04402F0AF
:10109B0090E000F0D297D29622121D281222AC12A9
:1010AB0016471216E574AA1217B2C2232290140126
:1010BB00E0B4400040028013B40A00400E900007D9
:1010CB00F0121EF974AA1217B2800574551217B2DA
:1010DB00C22322901401E0B40A0040028022FA7865
:1010EB000075A015F2121F84E0B43F005012B43209
:1010FB0000400DF2DAEF74AA1217B2121EF9800A31
:10110B00901500E4F074551217B2C22322780175C2
:10111B00A0149015467D20E2F0121F84DDF9121EFB
:10112B00F91222AC1216471216E574AA1217B2C2A4
:10113B00232290155CE0547FF56B901401E054076B
:10114B00F569901402E0B41B004002741AF56AC2F0
:10115B002322900009E054BF75F01E700375F01840
:10116B00B4010375F019901401E0B418004001E4C8
:10117B00901585F0901402E0B43C004001E490150A
:10118B0086F0901403E0B43C004001E4901587F026
:10119B00901404E0B5F0004001E4901588F0D23DC6
:1011AB00C22322901401E054BF700575F0188060C3
:1011BB00B4010575F0198058B4020575F01E805006
:1011CB00B4030575F01E8048B4040575F01E80400D
:1011DB007402900009F090150F7400F0A37400F0E6
:1011EB00A37400F0A37400F0A37418F0A37400F0C0
:1011FB00A37400F0A37400F0A37400F0A37400F0C8
:10120B00A37400F0A37400F074551217B2021310FC
:10121B00901401E0900009F0901402E0B418005013
:10122B00AF90150FF0F555901517F0901403E0B42F
:10123B003C00509C901510F0F556901518F090143A
:10124B0004E0B43C005089901511F0F55790151936
:10125B00F0901405E0B5F00040030211DB9015127D
:10126B00F0F55890151AF0C223901406E0B4180448
:10127B00D223800540030211DB901513F0F530905B
:10128B001407E0B43C0040030211DB30230560037C
:10129B000211DB901514F0F531901408E0B43C000A
:1012AB0040030211DB30230560030211DB9015159F
:1012BB00F0F532901409E0B5F00040030211DB3079
:1012CB00230560030211DB901516F0F53390140A19
:1012DB00E0A2E09222A2E19205A2E2921FA2E39287
:1012EB002AA2E4922BA2E5922DA2E6922EA2E792DD
:1012FB0013900008F0D296202204C2018002D20182
:10130B0074AA1217B2121EF91222AC121647121639
:10131B00E5122259C22322900009E054BF75F01E3A
:10132B00700375F018B4010375F019901401E0B453
:10133B00180040028047901402E0B43C0040028049
:10134B003C901403E0B43C0040028031901404E064
:10135B00B5F0004002802690151AF0901403E0902F
:10136B001519F0901402E0901518F0901401E0900C
:10137B001517F074AA1217B2121EF98005745512C4
:10138B0017B2C22322901401E0FA743F2AFA7902B1
:10139B00122189C22322901401E0FBA3E0FA9015DD
:1013AB0022E04AF0FAA3E04BF090E800F090E00066
:1013BB00EAF074AA1217B2C22322901401E0F4FBD4
:1013CB00A3E0F4FA901522E05AF0FAA3E05BF09058
:1013DB00E800F090E000EAF074AA1217B2C22322E0
:1013EB0090E800E0FB90E000E0FA74AA1217B2EB71
:1013FB001217B2EA1217B2C22322D201D29174AAE7
:10140B001217B2C2232220151720001DC23F302213
:10141B0018301F15301C04D201801D121C59800975
:10142B00103F028004D201800FD291C201C200C2D0
:10143B001574AA1217B2C22322202B04D200C29118
:10144B0074AA1217B2C22322302206C2AFD215D20F
:10145B00AF74AA1217B2C22322901401E0A2E09239
:10146B001D900008E092E3C21D5002D21DF075A042
:10147B0015781B901402E0F9F208A3E0FAF208A326
:10148B00E0F2FBC3740099748D9A74279B4003029E
:10149B0014B8C21D900008E054F7F090151B7400AF
:1014AB00F0A3F0A3F074551217B20214C0121EF978
:1014BB0074AA1217B2C22322900000E0FFFA12178F
:1014CB00B29000100FDF02804EE01217B22AFAA37F
:1014DB00E01217B22AFAA3E01217B22AFAA3E0120B
:1014EB0017B22AFAA3E0FDA3E0FEA3E0FCA3E0A35E
:1014FB001217B22AFAEC1217B22AFAC082C0838DE5
:10150B00828E830CDC028009E01217B22AFAA380C8
:10151B00F3D083D08280AEEA1217B2C223227F03AC
:10152B007E007A00903400E01217B22AFAA3DEF79D
:10153B00DFF59020007E10E01217B22AFAA3DEF737
:10154B00EA1217B2C223229015657F20E4F0A3DFC5
:10155B00FC756700C234C235C236901522E04402D6
:10156B00F090E000F074AA1217B2C22322E43035D7
:10157B000244013036024402FA1217B29015657F0D
:10158B0020E01217B22AFAA3DFF7EA1217B2C2232E
:10159B0022901401E0541F75F010A42400F582E58D
:1015AB00F03435F58375A0147801121D13A85E1263
:1015BB002252B4100040F89014011215F874AA12BC
:1015CB0017B2C223227C20EC1475F010A42400F572
:1015DB0082E5F03435F583E030E70FA85E12225236
:1015EB00B41000500280F61215F8DCDB22E0D2E7D3
:1015FB0075A018F2FB75A0177401F20875A018748A
:10160B0000F275A017F208A37A0DE075A018F22B63
:10161B00FB75A0177400F208A3DAEF75A018EBC3E3
:10162B0013F275A0177400F208885E75A08079021A
:10163B0074B5F375A08079057406F322122252B4A7
:10164B00080040F874BF855E82758318F0FB7583C4
:10165B00177401F074030582758318F02BFB7583E7
:10166B0017E4F0E430270274010582758318F02B20
:10167B00FB758317E4F0E52B0582758318F02BFBC4
:10168B00758317E4F0C082900009E054BFD0820547
:10169B0082758318F02BFB758317E4F0E535058213
:1016AB00758318F02BFB758317E4F0E53405827511
:1016BB008318F02BFB758317E4F00582758318EB09
:1016CB00C313F0758317E4F0058285825E90800268
:1016DB0074B5F09080057406F022122252B4080003
:1016EB0040F874BF855E82758318F0FB75831774A1
:1016FB0001F074200582758318F02BFB758317E4BA
:10170B00F0E430270274010582758318F02BFB750A
:10171B008317E4F0E52D0582758318F02BFB758399
:10172B0017E4F0C082900009E054BFD082058275A7
:10173B008318F02BFB758317E4F00582758318EB88
:10174B00C313F0758317E4F0058285825E908002E7
:10175B0074B5F09080057406F022FBE55EC3955DD1
:10176B00F4B403005003021766EBA85E75A018F2E1
:10177B0075A0177401F20875A018E5F0F22BFB7534
:10178B00A0177400F20875A018EBC313F275A0171D
:10179B007400F208885E75A080790274B5F375A0A9
:1017AB008079057406F322C0E0C082C08375831F65
:1017BB00855C82F0E55C04F583B55B072020FAD2EB
:1017CB009980F685835C202002D299D083D082D079
:1017DB00E02275A891C28CC28EC28F90305012023B
:1017EB0095903060120295903088120295C20BC210
:1017FB000DC212C20FC20CC210C20EC2078512114B
:10180B00758A00754C00752940752A01752EFF7578
:10181B002FFFC23875550075560075570075580067
:10182B0075330090151BE0F530A3E0F531A3E0F51F
:10183B0032C2AF75B80675A81FD246D28CD2AFC2D2
:10184B0023200D0820B5FD30B5FDB29412056F3085
:10185B00230D75A891C28CC28E120CA2021A6410B1
:10186B000C183004DCC2041203321207CA3001D147
:10187B0075A891C28CC28E021A64E539540375F0B7
:10188B000AA4F8E538540F28200E09B415B3D20E6C
:10189B007A0080ADF89018A8EA5403237380068071
:1018AB000A800E8028B816660A8096B817600A80E0
:1018BB0090B818030A808AB80054754618751278C8
:1018CB0075295BC2069030CB1202958046B8192859
:1018DB0075461E751296752915C2069030DD1202DB
:1018EB0095E53930E20AD2069030E6120295802354
:1018FB009030EF120295801BB800137546197512C4
:10190B007D75294DC2069030D41202958005C20E0A
:10191B0002184C90306E120295C2AF85434185443C
:10192B0042D2AFE54175F014A4F541A8F0E542753C
:10193B00F014A428F542754E00754D00D210D20F4D
:10194B00D294E539540375F00AA4F5F0E538540F39
:10195B0025F004F548F554E53B540775F00AA4F55A
:10196B00F0E53A540F25F0F549F553E53D5407756D
:10197B00F00AA4F5F0E53C540F25F0F54AF552E5D5
:10198B003F540375F00AA4F5F0E53E540F25F0F52E
:10199B004BF551D23AC202C218C21912056F30234D
:1019AB000302185D20100D75A891C28CC28E75288C
:1019BB0000021A64301902C219301843C2181207F8
:1019CB00CA30010A75A891C28CC28E021A64300DFE
:1019DB000B120AA790306E120295802390307B1267
:1019EB000295D296E5116017D51114D236C201C2F9
:1019FB0022900009E05440B4405F1220DB805A3043
:101A0B000247C202301603120AF0301B03120B639B
:101A1B001208D71223BD1203321202B9E554852ED8
:101A2B00F0B5F019852FF0B5F013900009E0544094
:101A3B00B440162038131220DBD2388002C238850E
:101A4B002EF085F02FE554F52E30170AC2173016FD
:101A5B0005C216120B210219A6D296901522E0444C
:101A6B0009F090E000F00201C5C21575A891901520
:101A7B0022E054FEF090E000F0903058120295C234
:101A8B008CC28EC23FC21AC218121C59204264204B
:101A9B00413A204025754618754000901554E0B426
:101AAB00E90C9030CB120295901554021B1190301B
:101ABB00C2120295901554021B119030D41202954C
:101ACB00901556754619754000021B113040129047
:101ADB0030DD12029590155A75461E754000021B9B
:101AEB00119030E612029590155875461E754004FC
:101AFB00021B119030EF12029590155875461E750A
:101B0B004000C240C241E0A3750F00F50EE0F50D99
:101B1B008000754700750936750C00750B0A750A40
:101B2B0001D209850E4FC2AF75B802E4C3954FF5CC
:101B3B008A202E0D90309B12029575A81BD28C809B
:101B4B005775A81FC28B9030601202959030B5125A
:101B5B00029520412F2040169030C212029574EA54
:101B6B00750F00F50E850E4F74C2F50D802A90305F
:101B7B00D4120295750F0074E0F50E850E4F749715
:101B8B00F50D801474BA750F00F50E850E4F74F0B9
:101B9B00F50D9030EF120295C246C28DC28FD2AFB7
:101BAB00C223D21C12056F302306120CA220012B6C
:101BBB0030020BC2021208D71203321202B93018CC
:101BCB00E3C2181207CA1223BD20010F30150AC237
:101BDB00929030A8120295800E80C975A891C28C84
:101BEB00C28E752800805512056F202314300226F3
:101BFB00C2021203321207CA301506200132201519
:101C0B0015D292202E0890309B1202958096903020
:101C1B00B5120295808E3018CEC21880CAD291753B
:101C2B00A891C28CC28ED201752800120CA2800C16
:101C3B00D29175A891C28CC28E752800901522E0A6
:101C4B004401F090E000F0D296C21C0201C5901541
:101C5B000FE0F555A3E0F556A3E0F557A3E0F558D3
:101C6B00A3E0F530A3E0F531A3E0F532A3E0F533C3
:101C7B00A330000390150FE0F54BA3E0F54AA3E06A
:101C8B00F549A3E0F548303D12901585E0F54BA3DF
:101C9B00E0F54AA3E0F549A3E0F548900009E054CC
:101CAB00BFB400087528007568048027B401087557
:101CBB002801756804801CB4030875280475680135
:101CCB008011B40408752802756801800675280315
:101CDB007568017536FC7537BFE54875F00A848564
:101CEB00F0384540F539E54975F00A8485F03AF549
:101CFB003BE54A75F00A8485F03CF53DE54B75F004
:101D0B000A8485F03EF53F227A108003121F84E28D
:101D1B00F0DAF9FAE0C39A70FB121F8422120DEB72
:101D2B00121EB0903440E0B4550D902000E0FCB48E
:101D3B00FE004006021DD5021E28902003E0A3F8EA
:101D4B00C3740098E0F8740C985003021DD59020D2
:101D5B000075A0007800ECF27D00FE121F84E0FB02
:101D6B00F2121F84E0FAF2121F847F0DE0F22CFCBA
:101D7B0074003DFD121F84DFF3BE0004D226804A9F
:101D8B00C226902010781075A0007F08E0F22CFC82
:101D9B0074003DFD121F84DFF3DEEF7E08E0F212CC
:101DAB001F84DEF9900003E0FFA3E0FE902800758E
:101DBB00A0087800EE4F6012E0F2121F842CFC7426
:101DCB00003DFD1FBFFFED1E80EA7F0F780075A061
:101DDB0015903400E0F2121F842CFC74003DFDDFE3
:101DEB00F37F0F780F75A015903410E0F2121F845B
:101DFB002CFC74003DFDDFF37F20784675A0159019
:101E0B003420E0F2121F842CFC74003DFDDFF3ED57
:101E1B008AF0B5F008EC8BF0B5F00280309015220B
:101E2B00E054FDF090E000F0D235C297C296122F2D
:101E3B00AE122FAED297D2967C209034FF7A1074CC
:101E4B0000A3F0DAFCE0B400FCDCF28010900000A0
:101E5B00E06006C226D2258004D226C2257D0478F6
:101E6B005590150FE0F6A308DDFA7D047830901538
:101E7B0013E0F6A308DDFA900008E0A2E09222A29C
:101E8B00E19205A2E2921FA2E3922AA2E4922BA274
:101E9B00E5922DA2E6922EA2E79213202204C20114
:101EAB008002D20122902FD775A00078007A10E41F
:101EBB0093F2121F84DAF8902FE775A01578007A49
:101ECB000FE493F2121F84DAF890300875A015789E
:101EDB000F7A0FE493F2121F84DAF8902FF275A0A9
:101EEB001578467A16E493F2121F84DAF82220262C
:101EFB0006202503120BCD120F50780075A0009011
:101F0B002000E2FC121D13EC7003021F4DC31304DF
:101F1B00FC121D13DCFB900003E0FCFFA3E0FD7A39
:101F2B0004EDC313FDEC13FCDAF7EF540F60010C57
:101F3B00BC0002800D780075A008902800121D13BC
:101F4B00DCFB780075A015903400121D13780F750B
:101F5B00A015903410121D13784675A015903420DF
:101F6B00121D13785675A015903430121D13903432
:101F7B00407455F0E0B455FC22A308B8000205A04C
:101F8B0022901537E0540F2323901F9873021FD90B
:101F9B0000021FF3000220DF00022134000221594E
:101FAB0000022165000221710002217D000221E85F
:101FBB00000222020002221C0002223700021FD85C
:101FCB0000021FD800021FD800021FD80022901554
:101FDB0037E05430FA334A5450FAA3E0543F90158B
:101FEB0024F0901525EAF022901538E0543FD2E703
:101FFB00FA901524E0F9901525E0F5F0301D048AD0
:10200B00588933122252B4050040F8758318855E47
:10201B0082EAF07583177401F005827583187401D9
:10202B00F02AFA7583177400F00582758318E5F0B2
:10203B00644003542045F0202207200D09440880FA
:10204B00053001024408F02AFA7583177400F00575
:10205B0082758318E9543FF02AFA7583177400F0E0
:10206B000582758318EA03547FF07583177401F0AA
:10207B00058285825E90800274B5F09080057406AF
:10208B00F0C22122122252B40300500280F6758353
:10209B0018855E82EAF07583177401F005827583EB
:1020AB00187408F02AFA7583177400F0058275838B
:1020BB0018EA03547FF07583177401F0058285824B
:1020CB005E90800274B5F09080057406F0C22122F8
:1020DB00743F8006C221901538E0543FD2E7FA12C4
:1020EB002252B40300500280F6758318855E82EA93
:1020FB00F07583177401F005827583187408F02A44
:10210B00FA7583177400F00582758318EA03547F00
:10211B00F07583177401F0058285825E90800274DE
:10212B00B5F09080057406F022901538E0543FFA14
:10213B00901526E0B40A02801204F0F9E58229F525
:10214B008274003583F583EAF0D21BC221229015ED
:10215B0038E0543FFA7918022189901538E0543F42
:10216B00FA7919022189901538E0543FFA791A024D
:10217B002189901538E0543FFA791B022189E562D9
:10218B00C39561F4B40500500280F375831C75A0F0
:10219B001B85628274FF4480FBF07401A882F205F8
:1021AB00827400F02BFB7400A882F20582E9547F45
:1021BB00F02BFB7400A882F20582EAF02BFB740073
:1021CB00A882F20582EB03547FF07401A882F2051A
:1021DB00828582629060057406F0C22122901537C9
:1021EB00E0232354C0F9A3E0543F49F9901522E0B2
:1021FB0049F090E000F022901537E0232354C0F90A
:10220B00A3E0543F49F9901523E049F090E800F022
:10221B0022901537E0232354C0F9A3E0543F49F42F
:10222B00F9901522E059F090E000F022901537E07C
:10223B00232354C0F9A3E0543F49F4F9901523E04C
:10224B0059F090E800F022E55EC3955DF4229060B2
:10225B00027415F0906000202D04741B800274131F
:10226B00F07407F0A3202D0474BB800274CCF090A3
:10227B0060047408F09060027405F09060057406B9
:10228B00F09080027415F0908000741BF07407F0CE
:10229B00A374CCF09080047408F09080057404F063
:1022AB0022901546E0A2E09203A3A3A3A3A3E0FA16
:1022BB005407239022C27341D241E641FA610E6169
:1022CB00226136614A614A7403904000F0740090B9
:1022DB004003F0752B00752D00807874049040003E
:1022EB00F07401904003F0752B00752D0180647420
:1022FB0005904000F07401904003F0752B00752D94
:10230B000280507406904000F07401904003F07509
:10231B002B00752D03803C7404904000F0740190E9
:10232B004003F0752B01752D048028740590400037
:10233B00F07401904003F0752B01752D058014741A
:10234B0006904000F07401904003F0752B01752D41
:10235B00068000EA5470C4239023677361876187FA
:10236B00618761876177617F6187618774049040C2
:10237B0001F0800E7405904001F0800674069040C9
:10238B0001F0EAA2E792959227900009E054BFB4BE
:10239B00000590154C8013B4010590154E800BB4BD
:1023AB0002059015528003901550E0F535A3E0F52A
:1023BB003422C0D0C0E0C0F0C082C083202D0E30CC
:1023CB00130BE562C39562F4B40800500302246E4C
:1023DB0075831C85628274FEF0F5F075831B7401A6
:1023EB00F0058275831C7400F025F0F5F075831BE6
:1023FB00E4F0058275831C7460F025F0F5F07583AD
:10240B001BE4F0058275831CE54BF025F0F5F075A8
:10241B00831BE4F0058275831CE54AF025F0F5F08B
:10242B0075831BE4F0058275831CE549F025F0F5F7
:10243B00F075831BE4F0058275831CE548F025F0ED
:10244B00F5F075831BE4F0058275831CE5F00354EE
:10245B007FF075831B7401F00582858262906005A5
:10246B007406F0D083D082D0F0D0E0D0D0222046BA
:10247B0003D28C32C0D0C0E0D214300D02B29674AD
:10248B0002C28CC58AD28CF54FE4C54C308D070443
:10249B0070027403C28DF550C3E54F948AE55094D6
:1024AB0000401BC3E529954FE52A95504004D208FF
:1024BB00801374B5954F74029550C2085007C20B28
:1024CB00C20D02259A30080D30070A200A28C207D0
:1024DB00054702259A200B71A208E53713F537E55E
:1024EB003613F536B4FC7EE537B4BF79300807D226
:1024FB000AD20702259A20B5FD30B5FDC294D2173A
:10250B007400B54808B54905B54A028016E53F5435
:10251B000775F00AA4F5F0E53E540F25F0F54BF5E1
:10252B0051D23A750938750B08750A08754700D2F0
:10253B000BC20AC207300F57754500754E00754D1B
:10254B0000D28ED28FC20F8046C000A208A809E627
:10255B0013F6D000D50A0E0509750A08D50B06C26D
:10256B000BD20DD20C300804D20780230547C207CB
:10257B00E54354F02544C4F50FE54F54F02550C402
:10258B00254350020544C3950FF54350021544D023
:10259B00E0D0D0322046030225B5C0E0054CE54C17
:1025AB007005D204754C03D0E032C0D0C0E0C0F04F
:1025BB00C082C083300911301507300504D29680D4
:1025CB0002B296C207022666C000A809E630E00EEA
:1025DB00301507300504D2968002B296D20703F667
:1025EB00D0000547E50AC333F50A506F750A01059C
:1025FB0009D50B67750936750B0A75470085485465
:10260B00854953854A52854B51D23AE54875F00AB4
:10261B008485F0384540F539E54975F00A8485F035
:10262B003AF53BE54A75F00A8485F03CF53DE54B00
:10263B0075F00A8485F03EF53FD28F302E1DD5689C
:10264B001AB209050CC28C758AFE756801E528540F
:10265B0007B40200502F756804802AB209850E4F0B
:10266B00E50CC3950D4002054F050CC28CE4C395D8
:10267B004F258AF58AD28C201A0BE509B43B06D27A
:10268B001AD218D294D083D082D0F0D0E0D0D032EE
:10269B00204603022900C0D0C0E0E54E6004154E71
:1026AB008019E54D601AC3E4954D754D00C28E251A
:1026BB008C5004D28E8009F58CD28ED0E0D0D032E3
:1026CB00C21AE545700D200D1320B5FD30B5FDC2C6
:1026DB00948009B40206D21AD294D218C0F0C083E7
:1026EB00C082200D03022828201A0C101406C20DDC
:1026FB00C20BD20F02282853A8FB854C17858A16CC
:10270B00E547A20785441485431543A8049211F5A8
:10271B00F0B4280040030227A6C3742895F023F5D4
:10272B00139415400BC20DC212C20BD20F022828F4
:10273B00E514C313C51513F51420110BC39516E53A
:10274B00159517400280021513E5148513F0A4F5B7
:10275B001685F017E5158513F0A42517C313C516B9
:10276B0013C516C313F517E51613F516E517C313A3
:10277B00F515E51613C515C313C51513F51425412A
:10278B00F541E5153542F542E5162541F54DE517C1
:10279B003542F54E154ED212022830942823F513EC
:1027AB009415400BC20DC212C20BD20F022828E5A2
:1027BB0014C313C51513F51420110BC39516E5158A
:1027CB009517400280020513E5148513F0A4F51646
:1027DB0085F017E5158513F0A42517C313C516133C
:1027EB00C516C313F517E51613F516E517C313F541
:1027FB0015E51613C515C313C51513F514C3E5411C
:10280B009514F541E5429515F542C3E5419516F54D
:10281B004DE5429517F54E154ED212800885424E66
:10282B0085414D154EE545B403028008B40102D233
:10283B00190228F0300D58301255901522E054F63D
:10284B00F090E000F0851211E539540375F00AA4FD
:10285B00F5F0E538540F25F0F548E53B540775F0D6
:10286B000AA4F5F0E53A540F25F0F549E53D540778
:10287B0075F00AA4F5F0E53C540F25F0F54A740009
:10288B00B54817B54914B54A110548054B80469014
:10289B001522E04408F090E000F00548E548B54605
:1028AB00347548000549E549B43C2A754900054A89
:1028BB00300610E54A75F00A84E5F06006740225CF
:1028CB0048F548E54AB43C0D754A00054BE54BB459
:1028DB001803754B00854854854953854A52854BDF
:1028EB0051D202D23A0545534503D082D083D0F062
:1028FB00D0E0D0D032C0D0C0E0C0F0C083C08230B6
:10290B00150302299E203D3D0548E548B5464A750D
:10291B0048000549E549B43C40754900054A30413A
:10292B001020400DE54A75F00A84C5F06003754828
:10293B0002E54AB43C23754A00054BE54BB4181924
:10294B00754B008014901585E0F54BA3E0F54AA379
:10295B00E0F549A3E0F548C23DE54BB53035E54A16
:10296B00B53130E549B5322BE548B53326D2913038
:10297B002B0D200506D215D23F8018D201801430C2
:10298B0000052005F680EE85554B85564A8557493F
:10299B00855848D202C21A20B5FD30B5FDC294D07D
:1029AB0082D083D0F0D0E0D0D032E564C39563857C
:1029BB00631BB407005006022E40022A4F122E4111
:1029CB00B4F0F7122E4120E779B47F78122E412014
:1029DB00E770B47F02800B2409F5F0900007E0B597
:1029EB00F062122E4120E75AB40259122E4120E711
:1029FB0051B410028008B430028003B47F46122E0B
:102A0B004120E73EF51AB40103022B13B402030273
:102A1B002B13B40303022B13B40403022B13B405BF
:102A2B0003022B13B41503022B8FB41603022B8F47
:102A3B00B41703022B8FB41803022B8FB4190502A2
:102A4B002A52151B022E3AE564C39563B41200504B
:102A5B0003022E40122E4120E7E8C3943075F00A92
:102A6B00A4F5F0122E4120E7D9C3943025F0B41809
:102A7B00004001E4901585F0122E4120E7C4B4000C
:102A8B00C3122E4120E7BBC3943075F00AA4F5F0B6
:102A9B00122E4120E7ACC3943025F0B43C0040012A
:102AAB00E4901586F0122E4120E797B40096122E73
:102ABB004120E78EC3943075F00AA4F5F0122E4135
:102ACB0020E73FC3943025F0B43C004001E490155F
:102ADB0087F0122E4120E72AB4002A122E4120E75C
:102AEB0021C3943075F00AA4F5F0122E4120E712A1
:102AFB00C3943025F0B41F004001E4901588F00218
:102B0B002B8F022A4D022A4FE564C39563B40F0045
:102B1B005003022E40122E4120E7E7C3943075F08C
:102B2B000AA4F51C122E4120E7D8C39430251CF5BE
:102B3B001C122E4120E7CBB400CB122E4120E7C252
:102B4B00C39430F51D122E4120E7B7B400B7122EF7
:102B5B004120E7AEC3943075F00AA4F51E122E4146
:102B6B0020E79FC39430251E75F00AA4F51E85F04F
:102B7B001F122E4120E78BC39430251EF51EE51F37
:102B8B003400F51F122E4130E750B4F750E51AB45C
:102B9B000104C2018076B403028071B40203022DDA
:102BAB005FB40403022CCFB40503022D17B4153008
:102BBB00D291C201201510200019C23F30221430CF
:102BCB001F11121C59800C103F028007C2AF121C40
:102BDB0059D2AFC200C215022DB0022E3A022A4DB5
:102BEB00B4160C3022EDC2AFD215D2AF022DB0B459
:102BFB001705D201022DB0B4180A202B04D200C243
:102C0B0091022DB0B41902D23D022DB0122252B452
:102C1B000500500280F6758318855E82E51C4480A2
:102C2B00F519B481004000F07583177401F005822B
:102C3B00758318E51DC3C23E9403400EF51D940326
:102C4B004004F51DD23E740D80027401F02519F578
:102C5B00197583177400F00582758318E51E33E52B
:102C6B001F3330E20244105413C51D600920E104E8
:102C7B00744080027420451DF51DE51AB4030674DB
:102C8B0008451DF51DE51D103E024408F02519F5FC
:102C9B00197583177400F00582758318E51E547F30
:102CAB00F02519F5197583177400F00582758318D3
:102CBB00E51903547FF07583177401F00582858243
:102CCB005E022DA4122252B40300500280F67583CB
:102CDB0018855E82E51C4480F519F0758317740125
:102CEB00F005827583187418F02519F5197583177B
:102CFB007400F00582758318E51903547FF0758312
:102D0B00177401F0058285825E022DA4122252B443
:102D1B000300500280F6758318855E82E51C4480A3
:102D2B00F519F07583177401F00582758318740F0C
:102D3B00F02519F5197583177400F0058275831842
:102D4B00E51903547FF07583177401F005828582B2
:102D5B005E022DA4122252B40300500280F675833A
:102D6B0018855E82E51C4480F519F0758317740194
:102D7B00F005827583187408F02519F519758317FA
:102D8B007400F00582758318E51903547FF0758381
:102D9B00177401F0058285825E90800274B5F09005
:102DAB0080057406F074F075831C856282F07400E4
:102DBB0075831BF00582E5616582607385826274A1
:102DCB007F75831C856282F0740075831BF005820E
:102DDB00E56165826059858262740375831C856227
:102DEB0082F0740075831BF00582E5616582603F9C
:102DFB00858262740275831C856282F07400758310
:102E0B001BF00582E5616582602585826274F7752A
:102E1B00831C856282F0740075831BF00582E5616B
:102E2B006582600B8582629060057406F080008578
:102E3B001B630229B52275831A851B82E0051B22B1
:102E4B00C0D0C0E0C082C08310990C109829D083E9
:102E5B00D082D0E0D0D032C299E55B655C7005C200
:102E6B0020022E7FD220855B82055B75831FE0F5E8
:102E7B00997598D0022E53E59975831E855A82F069
:102E8B0075831D209A04740080027401F0A3E55928
:102E9B006582600385825A022E53C0D0C0E0C08287
:102EAB00C083908005E030E103022F4B908005E05A
:102EBB0030E203022F96906005E030E103022EE032
:102ECB00906005E030E205022F1F80D6D083D082C0
:102EDB00D0E0D0D032E56165627009906005740472
:102EEB00F0022ECB202D1D9060027415F075831B04
:102EFB00856182E06008906000741FF0800690602E
:102F0B0000741BF075831C856182E0906003F005F3
:102F1B0061022ECB906001E075831985648220E5F8
:102F2B0004740080027401F0906003E075831A85CD
:102F3B006482F0A3E56365826003858264022ED50B
:102F4B00E55D655E700F9080057404F090800274EF
:102F5B00A5F0022EB79080027415F0758317855D6E
:102F6B0082E06008908000741FF0800690800074EF
:102F7B001BF0758318855D82E0908003F0055DB4CE
:102F8B008100400400000000022EB7908003E07522
:102F9B008316856082F0A3E55F658260038582609E
:102FAB00022EC17A3EEAC0E0122FBCD0E0FADAF56D
:102FBB00227A007B20DAFEDBFC227A007B0ADAFE27
:102FCB00DBFC227A007B32DAFEDBFC220000000005
:102FDB000000080A020200000000000000000000D0
:102FEB000000000000000000000100040047C7447F
:102FFB00E8397B396CEE00E5CDBECEBD000000009C
:10300B00001800000000000000008D27010144693A
:10301B00676974616C2042696E6C6F6F702000027F
:10302B0001496E697469616C697A696E672E2E2E1F
:10303B002000020156657273696F6E20362E303890
:10304B00202020200001015265616420000101470E
:10305B00656E20200001062D2D3A2D2D3A2D2D2E9B
:10306B002D2D0002014C6F636B6564202020200026
:10307B00020153656C662047656E202000020141FA
:10308B0077616974696E6720534D50544520200059
:10309B00020152756E6E696E672020200002014995
:1030AB00646C696E6720202020000201562D537935
:1030BB006E632020202000020B32332E393736006E
:1030CB00020B32342066707300020B3235206670AF
:1030DB007300020B33302066707300020B32392EF3
:0D30EB0039376400020B32392E39376E0080
:00000001FF
